:03218400750800DB
:20218A00C00D85810DE582FF24F850028032AE088FF005F07401800225E0D5F0FBFFE50DF8
:2021AA0024FDF8E66005EF42068005EFF4FF5206C006C0069000071221F11581D0068E0872
:2021CA00D00D22AF82C007C0079000071221F11581D0078F0822E4C0E09000041221F11505
:0721EA0081900002022207B0
:2021F100C00D85810DAD84758408E50D24FDF8E6F08D84D00D22AD84758408E0FE8D848E1C
:02221100822227
:2022130085828D438920438840759850C2AC22A298E433F58222858299C2993099FD221056
:20223300980280FB85998222AD82AE83AFF08D828E838FF0122455FC60180DBD00010E8CB2
:1322530082C007C006C005122229D005D006D00780DC2247
:0421000002212B325B
:01210B0032A1
:012113003299
:01211B003291
:0321230002228E07
:032187000221260C
:052126001223F380FE0E
:20226600750901750BFF750CFF750AFF22C2AFC2AC90247575F08012223B7582FF1221CDE8
:20228600122266D2AFD2AC22C020C0E0C0F0C082C083C007C006C005C004C003C002C0016C
:2022A600C000C0D075D00030993B74FFB50A028034E50A249C500875990A122266802474C6
:2022C600F6250A501575F00AE50A842430F59975F00AE50A8485F00A80097430250AF5995F
:2022E600750AAAC29920980302239EAF998F82C0071221CDD007C298BF3000500302236FAF
:20230600EF24C640647401B5090280077402B50953802974FFB50B08EF24D0F50B02239E6D
:2023260074F6250B4011E50B75F00AA4F50BEF24D0250BF50B8061122273805C74FFB50CFE
:2023460007EF24D0F50C805074F6250C4011E50C75F00AA4F50CEF24D0250CF50C803912EB
:2023660022738034122273802FBF2F057509028027BF3D21749C250B4016E50C6012749C78
:20238600250C400C850CF0E50B84F50AD29980081222738003122273D0D0D000D001D002EF
:2023A600D003D004D005D006D007D083D082D0F0D0E0D02032C00D85810DAE82AF837402FF
:2023C600F00EBE00010FE50D24FBF886040886058D048E828F83ECF0A3AE82AF83E50D245B
:2023E600FBF886058E828F83EDF0D00D227D8E7E227F80C005C006C0079020231223BB1587
:2024060081158115817582F41222131222661221E0AF82BFFF33C2AFC2AC122222E582600C
:20242600ED122232AF82BF300040E3EF24C640DEBF3000400C8F82C007122229D0071F8023
:0F244600EF75820A12222980C5D2AFD2AC80BFB7
:152475004D697374616B65206861732068617070656E640A001E
:06215A00E478FFF6D8FD59
:202138007900E94400601B7A0090248A780075A060E493F2A308B8000205A0D9F4DAF27540
:02215800A0FFE6
:202160007800E84400600A790075A060E4F309D8FC7800E84400600C7900906000E4F0A3BF
:04218000D8FCD9FAB4
:0D212B00758120122471E5826003022126D7
:1C24550020F71430F6148883A88220F507E6A88375830022E280F7E49322E02296
:04247100758200224E
:00000001FF
